:100000000C94BB040C94631F0C94D8040C94D80477
:100010000C94D8040C94D8040C94D8040C94D804F0
:100020000C94D8040C94D8040C94A4260C94762731
:100030000C946E210C94D8040C94D8040C94D8041D
:100040000C94D8040C94D8040C94D8040C94D804C0
:100050000C94D8040C9412220C94D8040C94D80458
:100060000C94D8040C94D8040C94D8040C94D804A0
:100070000C94D8040C94D8040C94D8040C94D80490
:100080000C94D8040C94D8040C94D8040C94D80480
:100090000C94D8040C94D8040C94D8040C94D80470
:1000A0000C94D8040C94D8040C94D804990799079C
:1000B000C507C5072D084B08630963095608EF08F3
:1000C00000090009E3270A2802290A2802295628DC
:1000D00079280229D028DF282B0014001A000800F4
:1000E00015001700000000000000290004001600A1
:1000F000070009000A00500000005100E0001D0048
:100100001B0006001900050003512A0028002A00E0
:10011000130012000C0018001C000000000000007A
:10012000340033000F000E000D000B004F000000E4
:100130005200E3003800370036001000110004516F
:100140002C62E6002B0014001A00090013000A00BC
:100150000000000000002900040015001600170030
:100160000700520000005100E0001D001B000600C7
:100170001900050003512C002A002A0033001C003E
:1001800018000F000D0000000000000034001200F5
:100190000C00080011000B004F0000005000E300AD
:1001A00038003700360010000E00045128004C00C3
:1001B0002B0034003600370013001C000000000044
:1001C0000000290004001200080018000C00520072
:1001D00000005100E000330014000D000E001B0071
:1001E00003512C002A002A000F00150006000A0007
:1001F00009000000000000002D001600110017008B
:100200000B0007004F0000005000E3001D00190024
:100210001A0010000500045128004C0035021E028F
:100220001F022002210222020000000000004C00F8
:100230003A003B003C003D003E00E00000000100B1
:100240000100400041004200430044000100010061
:1002500001002A00270226022502240223020000B0
:1002600000000000310230022F022E022D023F005A
:10027000E4000000010001004D00370036004A0094
:10028000450001000100010035001E001F00200094
:10029000210022000000000000004C003A003B005A
:1002A0003C003D003E000100000001000100400054
:1002B00041004200430044000100010001002A0007
:1002C0002700260025002400230000000000000075
:1002D000310030002F002E002D003F0001000000F3
:1002E000010001004E00370036004B0045000100C0
:1002F00001000100000000000000000000000000FC
:1003000000000000000000000000000000000000ED
:1003100000000000000000000000000000000000DD
:1003200000000000000000000000000000000000CD
:1003300000000000000000000000000000000000BD
:1007900000000000000000000100005C01000100FA
:1007A0000100010000000000000001000100295CC0
:1007B0001D5C1E5C135C01000000010001000100D3
:1007C00001000100010001000100010001004C00D6
:1007D0000100010001000100010000000000000014
:1007E00001000100A95DA85DA75D0A5C0100000091
:1007F0000100AE00AB00A900AA00A80001000100A2
:100800000100010042034D006F006E006B006500A7
:1008100065006200730020004F00720074006800E1
:100820006F0064006F0078002000520065007600C1
:100830002E003300200028005400650065006E0083
:100840007300790029000000200364006500640043
:100850007500630074006900760065006D006F002C
:100860006E006B00650065000000040309040902C6
:100870003B00020100A0FA0904000001030101008D
:100880000921110100012240000705810308000130
:1008900009040100010300000009211101000122E7
:1008A0007B00070582032000011201000200000006
:1008B00008EDFE603001000102000105010902A1FE
:1008C0000185020901A10005091901290815002562
:1008D000019508750181020501093009311581254D
:1008E0007F95027508810609381581257F95017568
:1008F000088106050C0A38021581257F95017508C7
:100900008106C0C005010980A101850319012AB72C
:1009100000150126B700950175108100C0050C096E
:1009200001A101850419012AA002150126A0029542
:100930000175108100C005010906A101050719E034
:1009400029E71500250195087501810295017508B3
:1009500081010507190029FF150026FF009506757E
:100960000881000508190129059505750191029571
:100970000175039101C011241FBECFEFDAE0DEBF85
:10098000CDBF11E0A0E0B1E0E0EAF3E502C00590E0
:100990000D92A23AB107D9F722E0A2EAB1E001C074
:1009A0001D92A33BB207E1F70E945F180C94CE2979
:1009B0000C9400000F9300E124E043E00E946C05DA
:1009C0000F910895FB01883A2DE5920761F0893A6D
:1009D0002DE5920769F0873A9D4591F4828188233D
:1009E00081F080E009C08281882359F081E004C051
:1009F0008281882331F082E00E94520580E00895D0
:100A000081E0089581E008950C94E20408950C9427
:100A100006051F93CF93DF9300D000D01F92CDB770
:100A2000DEB749835A836B833091A50189819A810E
:100A3000311114C0662359F0222349F00E94A00B03
:100A4000182F682F89819A810E94490B03C00E9448
:100A5000740B182F69817A81812F04C00E94A00B2A
:100A600069817A810F900F900F900F900F90DF9116
:100A7000CF911F910C94E712FC01262F40815181E8
:100A80006281738184810C94090581E00895CF937C
:100A9000DF93EC0160E00E943C05BE01DF91CF9145
:100AA0000C940705CF92DF92EF92FF92C12CD12CCC
:100AB0007601C39404C0CC0CDD1CEE1CFF1C8A958F
:100AC000D2F78C2D0E943C10C701B601FF90EF9029
:100AD000DF90CF900C944B0A8F929F92AF92BF926F
:100AE000CF92DF92EF92FF920F931F936B017C01E5
:100AF00081E090E0A0E0B0E04C015D0104C0880C12
:100B0000991CAA1CBB1C4A95D2F7AC01BD0104C0BC
:100B1000440F551F661F771F2A95D2F74829592978
:100B20006A297B2904C0880F991FAA1FBB1F0A9539
:100B3000D2F78A019B010C211D212E213F21401754
:100B400051076207730739F4BC01CD016C297D2977
:100B50008E299F290AC080959095A095B095BC01DB
:100B6000CD016C217D218E219F211F910F91FF903E
:100B7000EF90DF90CF90BF90AF909F908F900895AF
:100B80000C9457140C94531408950E94F3090E9476
:100B9000C4052FEF84E39CE0215080409040E1F7B2
:100BA00000C000000C9438220F931F93CF93DF9363
:100BB0008C0161E00E943C05EC01B8010E94040533
:100BC0008823F1F1B801CE010E94701E8823C1F183
:100BD000B801CE010E940D1B882391F1B801CE010E
:100BE0000E94CC1D882361F1F8018281882309F1DC
:100BF000CB358DE5D807C1F050F4C115FCE5DF0712
:100C000081F0CF3DDC45A9F40E94D61019C0CC3547
:100C1000EDE5DE0761F0CD35DD4559F40E941A108F
:100C200008C00E94C5050CC00E94231002C00E948B
:100C30002610C801DF91CF911F910F910C940205EE
:100C400080E0DF91CF911F910F9108950E94502174
:100C50000C943F060E9442060C94562108950C9471
:100C60002E0681E008950C9431060895CF93C82F85
:100C70000E942F068C2F0E943306CF91089580E0AA
:100C80000C9436060E948E200C9436060E948E200C
:100C90009091A401891721F08093A4010C94360649
:100CA0000895CF93DF93CDB7DEB72B970FB6F894A7
:100CB000DEBF0FBECDBF4F83588769877A878B878A
:100CC00061110E94660F9E012F5F3F4F86E0F90180
:100CD00011928A95E9F785E0FE013796D9010190D6
:100CE0000D928A95E1F789819A814C815D81452B2E
:100CF00031F09F3F31F491E08F3F19F403C091E050
:100D000001C090E090FF09C049815A816B817C81CC
:100D10008D819E810E94870E05C0C9010E944505F4
:100D20008111F2CF2B960FB6F894DEBF0FBECDBF68
:100D3000DF91CF910895FC01808191810E94E20BA7
:100D40000895CF93882309F455C0C82F8CEF8C0FDA
:100D5000813AF8F48C2F0E94831D81114BC06C2FB7
:100D600080910201909103010E94F220882349F0B2
:100D70006C2F80910201909103010E942A210E9410
:100D8000880F6C2F80910201909103010E9428210D
:100D90000CC080E28C0F883058F4C77081E001C02D
:100DA000880FCA95EAF70E94490FCF910C94880FDB
:100DB000EBE5EC0FE33040F4F0E0E05AFE4F8081C9
:100DC00090E0CF910C94BA20E8E5EC0FE73150F4B5
:100DD000F0E0EE0FFF1FEE5CFE4F80819181CF911E
:100DE0000C94D020CD3E30F08C2F0E94E418CF918F
:100DF0000C94B619CF910895882389F19CEF980F30
:100E0000913A40F4682F80910201909103010E9471
:100E10002A210DC090E2980F983058F4877091E025
:100E200001C0990F8A95EAF7892F0E944F0F0C9401
:100E3000880F9BE5980F933020F480E090E00C94AD
:100E4000BA2098E5980F973120F480E090E00C9458
:100E5000D0208D3E20F00E943F190C94B6190895C1
:100E60001F93CF93DF93182FEB010E94A1062097C9
:100E700041F08FE99FE00197F1F700C00000219752
:100E8000F6CF812FDF91CF911F910C94FC0689330F
:100E900019F060E070E002C060E570E00C9430078B
:100EA000882321F00E94490F0C94880F089588230D
:100EB00021F00E944F0F0C94880F0895CF92DF927B
:100EC000EF92FF920F931F93CF93DF937C01D62F66
:100ED000C72FFC011281058102950F700E943F0F00
:100EE0008823B9F01123A9F08C2F807F803421F062
:100EF00080E28D0F883068F08091870282FD09C002
:100F000082E00E94E80F0E943F0F91E0D82ED92680
:100F100001C0D12CCC2EC2948FE0C8228C2D90E041
:100F20008C30910508F0CFC1FC01EA5AFF4F0C94B8
:100F30005C298C2F807FCF70882311F0C295C07FF1
:100F4000112399F0CC2309F4AAC180E28D0F8830D7
:100F500010F0D11104C08C2F0E94490F03C08C2FB8
:100F60000E94590F0E94880F9AC18D2F0E94FC0683
:100F7000CC2309F4A8C180E28D0F883038F1DD233D
:100F800029F18C2F0E945F0F24C08C2F807FCF709F
:100F9000803211F0C295C07FDD2319F0D130A1F16C
:100FA0003DC08091870282FF17C0112349F0CC23F6
:100FB00029F08C2F0E94490F0E94880F80E070C199
:100FC00080E00E94FC06CC2309F47DC18C2F0E9496
:100FD0004F0F0E94880F77C1112371F0002341F059
:100FE000013031F40E94690F8C2B0E94710F6BC18C
:100FF0000E94690F8C2B1DC0002319F0013009F4E9
:1010000062C10E947E0F25C0112321F0063008F036
:101010005AC10EC0053008F056C11BC0112361F043
:10102000002331F0F701858180FF39C18F708583FE
:101030008C2F0E94500747C1002359F0D93309F083
:101040003FC1FFEF07EE13E0F15000401040E1F721
:1010500035C18C2F0E94570736C18C2F86958695F7
:10106000837019F0813061F02EC1112321F08D2F92
:101070009C2F937002C080E090E00E94BA202BC1A8
:10108000112321F08D2F9C2F937002C080E090E0FF
:101090000E94D02020C18D2F112319F00E94E41846
:1010A00002C00E943F190E94B61915C18C2F83708F
:1010B00009F047C011110BC12D2F229526952770DD
:1010C000220F220F6D2F6F70862F90E0A0E0B0E00E
:1010D000022E04C0880F991FAA1FBB1F0A94D2F7C3
:1010E000D4FF10C04FE050E060E070E004C0440F57
:1010F000551F661F771F2A95D2F74095509560952A
:10110000709503C040E050E0BA01C695C695C37023
:101110008A019B01082B192B2A2B3B2BC901B801F3
:10112000C23049F058F4C13019F00E945F0ACFC0B4
:101130000E944D0ACCC00E94710AC9C00E944B0A8D
:10114000C6C0112319F08C2F817001C086958823A9
:1011500009F4BDC02D2F229526952770220F220F4E
:101160006D2F6F70862F90E0A0E0B0E0022E04C0DB
:10117000880F991FAA1FBB1F0A94D2F7D4FF10C073
:101180004FE050E060E070E004C0440F551F661F60
:10119000771F2A95D2F7409550956095709503C0BA
:1011A00040E050E0BA01C695C695C3708A019B0124
:1011B000082B192B2A2B3B2BC901B801C23049F04F
:1011C00058F4C13019F00E94240B81C00E94120B08
:1011D0007EC00E94360B7BC00E94850A78C0CF700B
:1011E000112339F08C2F0E94AB0A8D2F0E945007DB
:1011F0006EC08D2F0E9457078C2F0E94CC0A67C0AB
:10120000D23F21F128F4D03F41F0D13FC1F043C09B
:10121000D33F19F1D43F79F03EC0112341F005309E
:1012200008F051C08C2F8F710E94F10A4CC006301B
:1012300008F049C0F7CF8091870282FF18C01123C0
:1012400039F08C2F8F710E94AB0A3DC01123C9F376
:101250008C2F8F710E94CC0A36C0112329F08C2F5D
:101260008F710E94960A2FC00E94910A2CC01123F0
:1012700049F0CF718C2F0E94AB0A63E08C2F0E9443
:10128000CD0F21C081E00E94E80F0230E0F082E043
:101290000E94E80F18C0112331F0002391F28D2F26
:1012A0000E94A10610C0002399F2D93349F41FEF20
:1012B00027EE33E0115020403040E1F700C000003D
:1012C0008D2F0E94FC0688EF8C0D843020F40E9444
:1012D0008E200E943606DD20C9F00E943B0F80FD63
:1012E00015C0F70112820E94350F0E94AB0AC70198
:1012F0000E94A7090E94350FDF91CF911F910F9196
:10130000FF90EF90DF90CF900C94CC0ADF91CF91BB
:101310001F910F91FF90EF90DF90CF9008950F9362
:101320001F93CF93DF93EC01688179818A810E94BA
:10133000ED0B8C010E94480B0E94390AB801CE01C6
:101340000E945E07DF91CF911F910F910895CF9377
:10135000DF93EC01988189812B813C81232B31F033
:101360008F3F31F481E09F3F19F403C081E001C059
:1013700080E080FD1DC0CE010E94D405811110C007
:101380000E943F0F8823A1F08A81882389F08091F1
:10139000870282FD0DC082E0DF91CF910C94E80FAF
:1013A000CE010E948F09CE01DF91CF910C944705A9
:1013B000DF91CF91089580E090E00E94BA2080E014
:1013C00090E00E94D0200E94660F0E94880F0E9429
:1013D000E71A0C94B61980910201909103010E94C2
:1013E0002C210C94DB090E94560F0C94EB0992956A
:1013F0009F70963079F010F4925001C09A5092305C
:1014000068F4803F69F018F4883E40F409C0843FD6
:1014100029F406C0883E20F0813F11F080E0089555
:1014200081E00895FC01808191810E94E20B0E947D
:10143000F7090895CF93DF9300D000D01F92CDB766
:10144000DEB70F900F900F900F900F90DF91CF911C
:101450000895CF93DF9300D000D000D0CDB7DEB792
:1014600026960FB6F894DEBF0FBECDBFDF91CF91A9
:101470000895089508950C943A0A0C943B0A0E942A
:101480003D0A6093CD017093CE018093CF0190937C
:10149000D0010C94DB090C943F0A0F931F93009129
:1014A000CD011091CE012091CF013091D001602B60
:1014B000712B822B932B1F910F910C943F0A0F934A
:1014C0001F930091CD011091CE012091CF01309159
:1014D000D00160237123822393231F910F910C94D9
:1014E0003F0A0F931F930091CD011091CE012091DF
:1014F000CF013091D00160277127822793271F9158
:101500000F910C943F0A0C94DA040E94830A6093B2
:10151000C9017093CA018093CB019093CC010C94C4
:10152000DB0960E070E0CB010C94850A0F931F93F8
:1015300041E050E060E070E08A019B0104C0000FD0
:10154000111F221F331F8A95D2F7C901B8011F91BD
:101550000F910C94850A0F931F9341E050E060E0D7
:1015600070E004C0440F551F661F771F8A95D2F79D
:101570008091C9019091CA01A091CB01B091CC0199
:101580008A019B01082B192B2A2B3B2BC901B8017F
:101590001F910F910C94850A0F931F9341E050E027
:1015A00060E070E004C0440F551F661F771F8A95E6
:1015B000D2F740955095609570958091C9019091B2
:1015C000CA01A091CB01B091CC018A019B010823F3
:1015D00019232A233B23C901B8011F910F910C94B1
:1015E000850A0F931F9341E050E060E070E004C073
:1015F000440F551F661F771F8A95D2F78091C90146
:101600009091CA01A091CB01B091CC018A019B01BC
:10161000082719272A273B27C901B8011F910F91D5
:101620000C94850A0F931F930091C9011091CA0170
:101630002091CB013091CC01602B712B822B932B0D
:101640001F910F910C94850A0F931F930091C9016C
:101650001091CA012091CB013091CC0160237123FC
:10166000822393231F910F910C94850A0F931F934C
:101670000091C9011091CA012091CB013091CC0198
:1016800060277127822793271F910F910C94850A59
:10169000089529E0929F800D1124E82FE695E695A4
:1016A000E695877051E001C0550F8A95EAF785E00D
:1016B000E89FF0011124EA55FE4F20E030E070E091
:1016C0004081CB01022E02C0969587950A94E2F7DD
:1016D0008170819584278523842781932F5F3F4FD5
:1016E0002530310569F7089529E0929F800D112476
:1016F000682F669566956695982F977085E0689F28
:10170000B001112440E050E080E0FB01E40FF51F40
:10171000EA55FE4F208130E0092E02C0369527950C
:101720000A94E2F721703327042E01C0220F0A9495
:10173000EAF7822B4F5F5F4F4530510531F708952F
:10174000BF92CF92DF92EF92FF920F931F93CF93AE
:10175000DF938C01C090C901D090CA01E090CB0109
:10176000F090CC018091CD019091CE01A091CF015C
:10177000B091D001C82AD92AEA2AFB2ACFE1D0E0C9
:10178000D701C6010C2E04C0B695A79597958795ED
:101790000A94D2F780FD04C0219790F7B12C07C0BE
:1017A000BC2EB8018C2F0E94FA120197A9F38B2D41
:1017B000DF91CF911F910F91FF90EF90DF90CF902D
:1017C000BF900895CF93DF93EC010E94A00BBE0160
:1017D0000E94FA12DF91CF9108951F93CF93DF9368
:1017E000EB019091A501992321F0CB010E94E20B1E
:1017F00013C0882349F0CB010E94A00B182F682F3B
:10180000CE010E94490B04C0CB010E94740B182F1B
:10181000BE01812F0E94FA12DF91CF911F9108958E
:101820001F93CF93DF93C091D10116E08091D20135
:10183000C81799F0D0E01C9FF0011D9FF00D1124F6
:10184000ED52FE4F40815181628173818481958187
:101850000E94290A2196C770E9CFDF91CF911F918D
:101860000895409103025091040260910502709125
:10187000060280910702909108020C94290AEF92C7
:10188000FF920F931F93CF93DF938091080282956D
:101890008F7009F065C080910502882309F460C04B
:1018A0008091D101F090D2011091030200910402C5
:1018B000609106027091070291E01F3F09F090E0ED
:1018C000C0910001D0910101292F96E0E92E8F15DA
:1018D00009F446C06115710521F00F3F21F030E099
:1018E00003C031E001C0322F90E030FD36C0E89EE9
:1018F000F001E99EF00D1124DF01AD52BE4F1196AB
:101900003C911197301329C03C91311326C0129697
:101910003C911297311121C013964D915C9114970F
:10192000461B570B4C175D07C0F4809108028F705F
:10193000806180930802E852FE4F80818F70806141
:10194000808383E092E00E94A709DF91CF911F91ED
:101950000F91FF90EF900C94100C01968770B7CF09
:10196000DF91CF911F910F91FF90EF9008959F927B
:10197000AF92BF92CF92DF92EF92FF920F931F939D
:10198000CF93DF93CDB7DEB761970FB6F894DEBF84
:101990000FBECDBF8C0185E0F801DE011D960190E0
:1019A0000D928A95E1F7D8011296EC90909103027E
:1019B000E0910402209106023091070221153105C1
:1019C00031F0EF3F31F481E09F3F19F403C081E033
:1019D00001C080E0B82FB1709B2E80FD47C1D801B7
:1019E0004C9111965C9111971396AD90BC90149701
:1019F00083E0C82E82E0D82EF0900502B501621B6C
:101A0000730B2091000130910101FF2009F4D9C02E
:101A1000809108026217730708F095C0282F207F75
:101A200009F052C05E1313C0491311C0FE2CE1101F
:101A30000EC08F708061809308020E94310CC60135
:101A40000E94A70980910802F80185834DC1AB2847
:101A500031F05F3F31F481E04F3F19F403C081E082
:101A600001C080E080FD03C081E08E2502C080E0DF
:101A700090E0F82FF170FF2E80FF1CC08091D10103
:101A80002091D20136E0821709F40BC190E0389F13
:101A9000F001399FF00D1124ED52FE4F6181561374
:101AA00006C06081461303C06281E61203C001963E
:101AB0008770E9CFFE2CEE2009F416C18091080250
:101AC00081608093080254C05E1306C0491304C0AD
:101AD000E11002C0F80199C0C8010E94120A8823CF
:101AE00061F1EE2051F120910802822F82958F70D2
:101AF00090E0029774F0809103029091040298871D
:101B00008F831986BB86AA862C87CE0107960E94F2
:101B1000A70986E0F801A3E0B2E001900D928A9552
:101B2000E1F70E943F0C0E94310C0AC05E1711F1D0
:101B3000C8010E94120A81112CC0C8010E94A70985
:101B4000FF24F394D1C0282F207F81F77A2DB98A02
:101B5000A88A6E2D89890E941A0A83E092E00E9469
:101B6000A70986E0D6011D928A95E9F70E94310CFB
:101B7000F12CBAC04913DCCFE110DACFF80185832C
:101B8000C8010E94A70986E0D6011D928A95E9F74F
:101B9000ABC0EE2091F220910802822F82958F70C7
:101BA00090E002970CF4B5CF80910302909104026B
:101BB0009A8389831B82BD82AC822E83CE010196DB
:101BC000A6CF6217730708F044C0FE2CEE2009F47C
:101BD000B4CF5E1330C049132EC02091080220FDFF
:101BE00021C0822F82958F70482F50E041155105FA
:101BF000C9F0F80125834F30510541F08F5F982FD0
:101C00009295907F822F8F70892B8583C8010E94C7
:101C1000A70986E0F801A3E0B2E001900D928A9551
:101C2000E1F73CC086E0F801A3E0B2E001900D923C
:101C30008A95E1F759C0C8010E94120A811169CF43
:101C400080910802816080930802C8010E94A70960
:101C50004BC07A2DB98AA88A6E2D89890E941A0AEA
:101C600086E0D6011D928A95E9F718C0EE2009F4A6
:101C700064CFC8010E94120AF82E882309F45DCFB0
:101C800086E0F801A3E0B2E001900D928A95E1F7B9
:101C900083E092E00E949B060E943F0C0E94310C60
:101CA00023C04D875E878D859E850E94E20B292F7C
:101CB00022952F70223028F49F7039F0811105C0D1
:101CC0000BC0243028F49F7049F4805E883020F0E7
:101CD000C8010E94A7099F2CF92C06C0D8011596AF
:101CE0009C91907F91F7F8CF8F2D61960FB6F89465
:101CF000DEBF0FBECDBFDF91CF911F910F91FF903F
:101D0000EF90DF90CF90BF90AF909F9008951F937A
:101D1000CF93DF93CDB7DEB72C970FB6F894DEBF25
:101D20000FBECDBF4F83588769877A878B879C8783
:101D3000CE0107960E94B70C8823D1F09F81888539
:101D40002A853B85232B31F08F3F31F481E09F3F83
:101D500019F403C081E001C080E080FD47C04F81DD
:101D6000588569857A858B859C850E94290A3EC0A5
:101D700086E0FE013796DE01119601900D928A955C
:101D8000E1F7FF81E8856A857B856115710531F092
:101D9000EF3F31F481E0FF3F19F403C081E001C05F
:101DA00080E080FD23C02091D20130E0C90101967E
:101DB000877099274091D10150E084179507F1F180
:101DC000F983EA837D836C8396E0929FD001939F91
:101DD000B00D1124AD52BE4FFE01319601900D920F
:101DE0009A95E1F78093D2010E94100C16E0809141
:101DF000D1019091D201891771F1189FC00111246E
:101E00008D529E4F0E94B70C882329F1E091D10199
:101E10001E9FF0011124ED52FE4F408151816281DD
:101E20007381848195810E94290A8091D10190E07B
:101E30000196877099278093D101D9CF0E94F30929
:101E40001092D2011092D101E3E0F2E086E0DF01CE
:101E50001D928A95E9F72C960FB6F894DEBF0FBE57
:101E6000CDBFDF91CF911F9108958091110285958B
:101E700085958595089580911102877008959091B8
:101E80001102977081E009F480E0089580911C02AE
:101E9000089590911C02892B80931C0208958095CF
:101EA00090911C02892380931C02089510921C02B9
:101EB000089590911B02892B80931B0208958095B1
:101EC00090911B02892380931B02089510921B029C
:101ED000089580911202089508950C946C0F0C944B
:101EE0006D0F9091870292FD08C090911202981791
:101EF00021F0809312020C946F0F089580911202CA
:101F0000882329F01092120280E00C946F0F08953C
:101F1000CF93DF93E0910201F091030180911C02C5
:101F20008083E0910201F0910301908180911B0276
:101F3000892B808380911202882381F0E091020135
:101F4000F09103019081892B80838091020190910F
:101F500003010E94E62081110E947E0FC0910201C0
:101F6000D091030148E050E069E072E0CE010E94A8
:101F70007629892B69F088E0FE01A9E0B2E00190A2
:101F80000D928A95E1F7CE01DF91CF910C94A120BB
:101F9000DF91CF9108950C946C0F9091870292FD80
:101FA00010C098E0899F90011124262B20931102E4
:101FB0000E94AB0A809111028595859585950C94B8
:101FC000CB0F0C94AB0A1092110280E00C94CB0F53
:101FD000209111028095822380931102982F97708F
:101FE00099F430E0482F082E000C550B24173507C4
:101FF00059F09091870292FD07C08595859585954A
:102000000E94CC0A0C94E30F08959091870292FBF2
:10201000222720F9281769F080FB92F99093870214
:1020200080918602909187020E94521082E00C9467
:10203000E80F08958091870282FB882780F991E05C
:1020400089270C94051081E00C94051080E00C9415
:10205000051080E090E00E94942921E0893E9E4F87
:1020600009F020E0822F089582E090E00C948C2902
:1020700083E090E00C948C29682F83E090E00C942E
:102080009A29CF9384E090E00E948C29C82F82E2A5
:1020900090E00E948C292C2F30E0A901582BCA0116
:1020A000CF910895CF93C92F682F84E090E00E94CC
:1020B0009A296C2F82E290E0CF910C949A29AB017F
:1020C000BC018FE090E00C94AC29AB01BC0183E132
:1020D00090E00C94AC2960E070E0CB010C946510AA
:1020E00060E070E0CB010E945F100C946B1069EE11
:1020F0007EEF80E090E00E94B82960E082E090E00E
:102100000E949A2960E083E090E00E949A29109250
:10211000CD011092CE011092CF011092D00160E05B
:1021200084E090E00E949A2960E082E290E00E94C0
:102130009A2960E085E090E00E949A2960E086E0BC
:1021400090E00E949A296FEF87E090E00E949A2920
:1021500040E050E0BA0188E090E00E94AC2960E0E5
:102160008DE090E00E949A2940E050E0BA0188E1B9
:1021700090E00E94AC2960E087E190E00E949A29FB
:1021800040E050E0BA018CE190E00E94AC2960E0B0
:1021900070E080E290E00E94B82940E050E0BA018F
:1021A00088E190E00E94AC290C9470100C94771098
:1021B0008EE090E00E948C2991E0811101C090E0B6
:1021C000892F0895682F8EE090E00C949A290E9440
:1021D000DB2160932D0270932E0280932F02909347
:1021E00030026093290270932A0280932B0290930D
:1021F0002C02089585B7806885BF85B7806885BF44
:1022000008950C94261608950C9403110C94031150
:102210000C9406110C9403110C940A110C940311E4
:102220000E94FA1087E194E10E9484200E940E111E
:102230000C940C110E9404110C9403110E941A14A6
:102240000C9435060E94C6210E94D6130E943E16A9
:102250000E946C150E941E110E94F51A0E944816D9
:102260000C9408115F926F927F928F929F92AF921F
:10227000BF92CF92DF92EF92FF920F931F93CF9373
:10228000DF93CDB7DEB72A970FB6F894DEBF0FBE47
:10229000CDBF0E949015C82E81110E94E7103DE12C
:1022A000832E32E0932E00E010E0502E802F0E940B
:1022B0003E145C01F401619071904F01682679260B
:1022C00061147104B1F40F5F1F4F0630110569F7F7
:1022D0008FEF89838A831B820E94CF218160782FB0
:1022E0009D838C8349815A816B818D810E94510627
:1022F0003AC08091310281FD0E944714D12CEE2416
:10230000E394F12CC3018E219F21892B29F10E9496
:1023100001118823A9F0DE825F82AE20BF2081E018
:10232000AB2809F480E088870E94CF218160782F54
:102330009A8789874E815F8168858A850E945106C8
:10234000000F111FF801E35EFD4F80819181E826A7
:10235000F926F182E08207C0D394EE0CFF1CF9E06D
:10236000DF12D0CFB0CF81E0C11001C080E02A964B
:102370000FB6F894DEBF0FBECDBFDF91CF911F9196
:102380000F91FF90EF90DF90CF90BF90AF909F9014
:102390008F907F906F905F9008950E9432110E94FD
:1023A00026160E94D4190C944606CF93DF930E9400
:1023B000FF12EC01811521E5920708F045C0811557
:1023C00030E5930708F094C0883E910528F5803EDB
:1023D000910508F0F8C0883A910570F4853A9105A6
:1023E00008F07CC08130910509F475C008F4E8C09C
:1023F000049708F0E8C0E4C08F3B910508F0E0C006
:10240000C85AD0E0CC0FDD1FCD59DE4F0990D881DE
:10241000C02DCE019464D8C0811540E2940758F4D1
:10242000811551E0950708F0CEC08D3E910508F466
:10243000C7C09065C9C0C11580E4D80708F4C0C002
:10244000DF70CE01906AC0C0811525E59207A8F41F
:10245000811534E5930708F095C0811543E594078D
:1024600008F07BC0811552E5950708F061C0D82FB0
:10247000CC27CE01816F906AA7C0C11589E5D80726
:10248000A0F4C11528E5D20708F082C0C11536E5D1
:10249000D30708F095C08C2F0E9493138F7190E0A2
:1024A000D82FCC27CE0190628FC0C1154AE5D40742
:1024B00008F474C0CE0190568115904208F080C097
:1024C0008D2F8F710E949313DD27D0628F71AE0123
:1024D000582BCA0179C081E090E076C0C55AD0E09F
:1024E000CF56DE4F8881C82FD0E0CE0190646CC0FB
:1024F00074E0969587957A95E1F7282F23703C2F05
:10250000337081E090E002C0880F991F3A95E2F79E
:102510009C68AC01522B9A019C2F9F7096959695C2
:1025200050E2959FE0011124C9018C2B9D2B4CC0DA
:102530008370992721E030E002C0220F331F8A9573
:10254000E2F79C2F9695969580E2989FE0011124E2
:10255000C22BD32BCE019C6837C08370992721E012
:1025600030E002C0220F331F8A95E2F79C2F969528
:10257000969540E2949FE0011124C22BD32BCE010B
:102580009A6822C0D82FCC27CE01846F906A1CC0D5
:10259000DC2FCC27CE01806F906A16C08C2F8F70F5
:1025A0000E94931394E0D695C7959A95E1F7CF7062
:1025B000D0E0DC2FCC27D0699E01282BC90104C0B4
:1025C00080E090E001C0CE01DF91CF91089526E335
:1025D000829FC0011124FC0129E0729FE00DF11DD2
:1025E0001124E60FF11DEE0FFF1FE852FF4F8591FA
:1025F000949108950E94E7120E94D511089582389F
:10260000910569F1B0F48133910509F46DC048F486
:102610008932910509F463C08A32910509F469C0D1
:1026200008958533910509F455C089339105B9F0B2
:102630000895833E910569F138F4803E9105B1F02B
:10264000823E910509F10895863E9105A9F1873EE4
:102650009105B9F1843E910509F064C023C0209131
:10266000860220FD4FC021FD4DC008958091860255
:1026700080FD44C08091870280FF44C08091860223
:1026800084FD42C083EE4DC08091860282FF38C037
:10269000F5CF8091860282FD33C08091870280FD54
:1026A00031C0ECCF8091870281FF32C080918602D9
:1026B00084FD2AC087EE35C08091860283FF26C044
:1026C000F5CF8091860283FD21C08091870281FD34
:1026D0001FC0ECCF8091860285FD1CC01DC080917B
:1026E000860285FD19C016C08091860286FD16C03F
:1026F00017C08091860286FD13C010C089E311C007
:1027000082EE0FC080EE0DC080E00BC086EE09C0E7
:1027100084EE07C089E205C085E303C08AE201C0F8
:1027200081E390E008959091860292FF0DC0282FDA
:102730002871283019F4877F846006C0282F2471FF
:10274000243011F48B7F886093FF0DC0282F2871EF
:10275000283119F4877E846106C0282F2471243122
:1027600011F48B7E88612091870220FF0DC0382FE5
:102770003871383019F4877F816006C0382F317185
:10278000313011F48E7F886021FF0DC0282F287111
:10279000283119F4877E816106C0282F21712131EB
:1027A00011F48E7E886194FD877E089510928202D6
:1027B0001092830210928402109285020895CF92A3
:1027C000DF92EF92FF926B017C010E94261681112D
:1027D0000EC00E94DB21C61AD70AE80AF90AC09285
:1027E0008202D0928302E0928402F0928502FF90EE
:1027F000EF90DF90CF9008950F931F930E942616BD
:10280000882321F01F910F910C94DB210E94DB2182
:1028100000918202109183022091840230918502FE
:10282000600F711F821F931F1F910F91089580E009
:10283000089508950E942910811102C00E94D610A7
:102840000E943410809331020E94411090938702BD
:10285000809386020E9419140E943810682F70E03D
:1028600080E090E00E944B0A6091C9017091CA011A
:102870008091CB019091CC010C94830AE82FF0E079
:10288000EE0FFF1FEB56FD4F808191810895089553
:1028900080EA8A95F1F7089500C008950C944814D1
:1028A00008950C9450140C9451140C9450140C94DE
:1028B00055140C945014FF920F931F93CF93DF93F2
:1028C00000D000D000D0CDB7DEB70E9426166091B0
:1028D000A102882309F443C056E0F52E8E010F5F54
:1028E0001F4FF8018F2D11928A95E9F7862F90E0FE
:1028F000880F991FB8018B569D4F0E94561688234A
:1029000099F08091880290E0880F991F46E050E08E
:10291000B8018B569D4F0E94762921E02093320208
:10292000892B61F410E018C0809132028823D1F322
:10293000F8011192FA94E9F710923202A0918802FC
:10294000B0E0AA0FBB1FAB56BD4F86E0F801019067
:102950000D928A95E1F711E00E94C20511C08091A5
:10296000880270E0660F771F6B567D4F90E0880FEE
:10297000991F8B569D4F0E94E0160E94591410E03B
:10298000812F26960FB6F894DEBF0FBECDBFDF9124
:10299000CF911F910F91FF900895F894E82FE29541
:1029A000EF70F0E031A1282F2F7081E090E001C09E
:1029B000880F2A95EAF7982F9095932391A392A1D7
:1029C000892B82A378940895CF93DF9380E30E94AC
:1029D000CD1486E60E94CD1487E60E94CD14C4E98A
:1029E000D1E089918F3F11F00E94CD1481E0CD3963
:1029F000D807B9F7DF91CF910895BF92CF92DF92B8
:102A0000EF92FF920F931F93CF93DF938C01C62F0A
:102A1000D0E0CE0183569E4F6C01FC0190819F3F18
:102A200009F450C0B62EF894E92FE295EF70F0E06B
:102A300081A19F7021E030E001C0220F9A95EAF752
:102A4000822B81A382A12095282322A378940E941F
:102A50004C14E4E9F1E04DE951E021E030E0E12CF3
:102A6000F12C61916F3F89F0A62FA295AF70B0E075
:102A700090968C9190E06F7002C0959587956A95BD
:102A8000E2F780FD02C0C90102C080E090E0E82AC0
:102A9000F92A220F331F4E175F0719F7F6018081BD
:102AA0008F3F11F00E94CD1461E0E114F10409F4AC
:102AB00060E08B2D0E944E14CC0FDD1FC00FD11F84
:102AC000F982E882DF91CF911F910F91FF90EF90F3
:102AD000DF90CF90BF900895809104018091040110
:102AE000811102C093E001C090E09093A10283E0C5
:102AF000891B809388020E94E4148CE0E5E9F2E0EF
:102B0000DF01982F1D929A95E9F7E9E8F2E0DF01DD
:102B10001D928A95E9F783E00E94E9150C94C0059F
:102B2000EF92FF920F931F93CF93DF93CDB7DEB752
:102B30002C970FB6F894DEBF0FBECDBF8E010F5F8E
:102B40001F4F8CE0F80111928A95E9F760E0C80107
:102B50000E94FD1461E0C8010E94FD1462E0C801FA
:102B60000E94FD144CE050E0B80189E892E00E9418
:102B700076297C0121E0892B09F420E0E114F1049D
:102B800041F08CE0F801A9E8B2E001900D928A953D
:102B9000E1F76091A10270E0660F771F6B567D4FE1
:102BA00043E089E892E00E94EA15EF2819F40E94B8
:102BB0005B1402C081E090E02C960FB6F894DEBF63
:102BC0000FBECDBFDF91CF911F910F91FF90EF907E
:102BD00008950895FF920F931F93CF93DF93F82EDC
:102BE000092F162FD72FC42F222349F081E080937D
:102BF00035020E94CF21909334028093330280915A
:102C000035028823D9F080913302909134020E94DA
:102C1000E721059798F0EF2DF02FA12FBD2F80E031
:102C200090E04C2F50E08417950734F421913191B6
:102C30002D933D930196F7CF10923502DF91CF91FE
:102C40001F910F91FF9008950C94D8108091380235
:102C500081110DC00E943B29811102C082E001C098
:102C600081E080933802823011F40E94362981E09D
:102C700090913802913009F080E008950E94241666
:102C8000809304010E94261681110C948E160895DB
:102C90000E942616811102C00C949016089581E0BE
:102CA000909139029A3008F080E008950F931F93B5
:102CB000CF93DF93EC018B01809139028A3038F495
:102CC000B801CE010E94DE1681111DC00AC080919C
:102CD0003602909137020E94E721843F914080F7AD
:102CE00015C0809139028F3F19F08F5F80933902B0
:102CF000809139028A3060F00E94CF219093370290
:102D00008093360203C01092390202C080E001C0F5
:102D100081E0DF91CF911F910F9108950C941D1FB9
:102D20000C94201FDF92EF92FF920F931F93CF938B
:102D3000DF937901C82F880FDD0B41155105A9F0EC
:102D4000FE0193E0EE0FFF1F9A95E1F7EB5FFE4F58
:102D500081819281865C9D4F208130E0421753072C
:102D600008F49A01A9010E948329CE010E9409203A
:102D7000D82E8823D1F001151105B9F083E0CC0FCE
:102D8000DD1F8A95E1F7FE01EB5FFE4F438150E0C6
:102D90000417150708F4A801CB5FDE4F6C817D8115
:102DA000665C7D4FC7010E9483298D2DDF91CF91F5
:102DB0001F910F91FF90EF90DF9008950C94FD17F5
:102DC0000C9419180F931F93CF93DF9300D000D06A
:102DD000CDB7DEB7609153027091540280915502D5
:102DE000909156020E94F621643671058105910585
:102DF00028F10E94FC13DC01CB010296A11DB11D3C
:102E000089839A83AB83BC8300E010E020E030E04C
:102E100044E050E0BE016F5F7F4F82E00E94921657
:102E2000182F882361F00E94DB2160935302709376
:102E30005402809355029093560201C011E0812FF5
:102E40000F900F900F900F90DF91CF911F910F91E6
:102E50000895AF92BF92CF92DF92EF92FF920F93BD
:102E60001F93CF93DF937C015B016A010E944F1691
:102E7000811103C001E010E002C00AE010E0C1E0EF
:102E8000D0E0F894B501C701F60109957894811155
:102E900015C021960C171D0794F0CC9F9001CD9F73
:102EA000300D300D112480E090E045E34A95F1F7B4
:102EB0000000019682179307C1F7E3CF81E0DF910D
:102EC000CF911F910F91FF90EF90DF90CF90BF9027
:102ED000AF900895AF92BF92CF92DF92EF92FF92A0
:102EE0000F931F93CF93DF93CDB7DEB727970FB61E
:102EF000F894DEBF0FBECDBF7B01C090A001D09083
:102F0000A10101E010E09E01295F3F4F40E050E049
:102F100060E070E080E00E949216182F882309F488
:102F20003EC056018FEFA81AB80A60914F02709107
:102F3000500280915102909152020E94F621643613
:102F400071058105910518F106E010E09E012F5FE3
:102F50003F4F40E050E060E070E081E00E94921658
:102F6000182F66E070E0C5010E94F61A91E02F81EB
:102F7000281390E0192339F10E94DB2160934F025E
:102F800070935002809351029093520211C066E0F8
:102F900070E0C5010E94F61A9F818913D5CF86E0A3
:102FA000F6013196DE01119601900D928A95E1F7B6
:102FB000112349F086E0FE013196A9E4B2E00190C8
:102FC0000D928A95E1F786E0E9E4F2E0D7010190FD
:102FD0000D928A95E1F7812F27960FB6F894DEBF00
:102FE0000FBECDBFDF91CF911F910F91FF90EF905A
:102FF000DF90CF90BF90AF9008950F931F93CF9322
:10300000DF93EC018B014AE657E10E9429178823E0
:1030100051F042EE56E1B801CE01DF91CF911F9100
:103020000F910C94291780E0DF91CF911F910F91A0
:1030300008950F931F93CF93DF93F894C091A0014D
:10304000D091A101CE01019626E0FB01DC010190A7
:103050000D922A95E1F766E070E00E94F61A8883E7
:103060007894F8946F81788589859A8500914502D6
:103070001091460220914702309148026017710773
:103080008207930751F06093450270934602809344
:103090004702909348020E94DF137894DF91CF910A
:1030A0001F910F9108950E94FC230E9422110C94FD
:1030B00008240E940C240E94CD110C9426240E9406
:1030C0006D210E94E3230E9410110E9453180E9458
:1030D00059180E941A11FBCF80915D0280FF06C033
:1030E0006091220170E0660F771F26C081FF04C047
:1030F0006091220184E005C082FF07C06091220137
:1031000088E0689FB001112417C090915C02992358
:10311000D1F060912101961788F72091220188E073
:10312000289F90011124929FA001939F500D11247C
:1031300070E0CA010E9448296038710540F46115A9
:10314000710519F406C068E070E0862F08958FE7D6
:10315000089581E0089580915D0280FF08C060912C
:103160001E0170E0759567957595679521C081FF83
:1031700006C060911E0170E07595679519C082FFC9
:1031800004C060911E0170E010C090915B02992311
:1031900099F060911D019617A0F780911E01899FFB
:1031A000C001112470E00E9448296038710540F484
:1031B0006115710519F406C061E070E0862F08956D
:1031C0008FE7089581E008958D3E21F40E946C18E8
:1031D000819504C08E3E29F40E946C188093610290
:1031E00008958F3E21F40E946C18819504C0803FA1
:1031F00029F40E946C18809360020895893F19F4A5
:103200000E94AB1805C08A3F31F40E94AB1881952B
:103210008093620208958B3F21F40E94AB18819540
:1032200004C08C3F29F40E94AB1880936302089578
:103230009FE0980F983078F421E030E0A90102C0B7
:10324000440F551F9A95E2F7CA0190915F02892BAE
:1032500080935F0208958D3F21F480915D0281602B
:103260000BC08E3F21F480915D02826005C08F3FCC
:1032700029F480915D02846080935D0208958D3E03
:1032800039F49091610297FF35C01092610259C0E4
:103290008E3E29F4909161021916BCF32BC09091D7
:1032A00060028F3E29F497FF25C01092600249C04A
:1032B000803F19F41916CCF31DC090916202893F2A
:1032C00029F41916BCF4109262023BC08A3F19F42B
:1032D00097FF10C0F8CF8B3F39F49091630297FFAE
:1032E00009C0109263022DC08C3F21F490916302BB
:1032F0001916BCF39FE0980F983080F421E030E07D
:10330000A90102C0440F551F9A95E2F7CA018095A2
:1033100090915F02892380935F0213C08D3F21F457
:1033200080915D028E7F0BC08E3F21F480915D0203
:103330008D7F05C08F3F29F480915D028B7F809344
:103340005D0280916002811106C08091610281114D
:1033500002C010925C0280916202811106C08091CD
:103360006302811102C010925B0208950E94CF2176
:1033700020916002211104C020916102222321F0DA
:1033800090935A028093590220916202211104C045
:1033900020916302222321F09093580280935702D8
:1033A0008EE592E00C94AC20EF92FF920F931F9366
:1033B000CF93DF9300D000D000D0CDB7DEB786E04A
:1033C000EEE5F2E0DE01119601900D928A95E1F7AB
:1033D000E0906002F090610200916202109163023D
:1033E00010926002109261021092620210926302C7
:1033F000E11003C0FF2009F45DC080915902909153
:103400005A020E94E721AC0190915C02992339F0A5
:103410002091230130E02417350758F04BC020914C
:1034200024018AE0289F900111242417350718F001
:1034300041C09F3F19F09F5F90935C02EE2061F0C6
:103440000E946C181E1414F09FEF01C091E0989F29
:10345000902D112490936002FF2061F00E946C185F
:103460001F1414F09FEF01C091E0989F902D11243C
:1034700090936102309160023323E1F02091610268
:103480002223C1F045EB3403C0011124992319F024
:103490009093600203C081E08093600235EB2303C8
:1034A000C0011124992319F09093610203C081E0B7
:1034B00080936102011103C0112309F45DC0809162
:1034C0005702909158020E94E721AC0190915B0253
:1034D000992339F020911F0130E02417350758F067
:1034E0004BC0209120018AE0289F900111242417CD
:1034F000350718F041C09F3F19F09F5F90935B0222
:10350000002361F00E94AB18101614F09FEF01C069
:1035100091E0989F902D112490936202112361F005
:103520000E94AB18111614F09FEF01C091E0989F14
:10353000902D112490936302309162023323E1F0C5
:10354000209163022223C1F045EB3403C001112412
:10355000992319F09093620203C081E08093620284
:1035600035EB2303C0011124992319F090936302D2
:1035700003C081E0809363028091600281110BC0DF
:1035800080916102811107C080916202811103C0A4
:103590008091630281110E94B619EB82FC820D8337
:1035A0001E8386E0FE013196AEE5B2E001900D92F9
:1035B0008A95E1F726960FB6F894DEBF0FBECDBF11
:1035C000DF91CF911F910F91FF90EF900895EEE55D
:1035D000F2E086E0DF011D928A95E9F710925C0225
:1035E00010925B0210925D0208950895FC01680F2D
:1035F000791F8FEF91E3E617F70771F0219182278A
:1036000028E030E087FF03C0880F892701C0880FBA
:1036100021503109B9F7EFCF0895CF93DF93EC0133
:10362000FB018281882309F43CC1C430FDE5DF073A
:1036300060F4CB3F9CE5D90788F49E0122503C45BD
:103640002431310508F02EC109C0C236EDE5DE0790
:1036500029F0C63AFDE5DF0709F024C10E944110B8
:103660009093870280938602C1318CE5D80709F4D4
:10367000C6C008F042C0C930ECE5DE0709F49BC0C3
:1036800000F5C5308CE5D80709F485C078F4C3305F
:10369000ECE5DE0709F478C008F07AC0C230DC45FA
:1036A00009F0F5C0809186028160EFC0C7309CE5CB
:1036B000D90709F478C008F07AC080918602806149
:1036C000E4C0CD30FCE5DF0709F487C058F4CB3007
:1036D0009CE5D90709F479C008F07BC08091860287
:1036E00088606FC0CF30FCE5DF0709F480C008F0C8
:1036F00082C080918602877FC8C0CE3F9CE5D907F3
:1037000009F471C000F5C531FCE5DF0709F485C097
:1037100068F4C3319CE5D90709F475C008F095C079
:103720000E94F309809186028F77AFC0CC3FFCE501
:10373000DF07A9F108F054C0CB3FDC4509F0A7C072
:103740008091870240C0C230EDE5DE0709F489C0F0
:1037500058F4C1158DE5D80709F45AC008F069C0BE
:103760008091870282602FC0C236EDE5DE0709F442
:103770007CC0C63AFDE5DF0709F481C0C330DD45F2
:1037800009F085C080E06EC08091860282607DC0B5
:103790008091860216C080918602886076C08091F2
:1037A000870282604FC08091860280626EC08091E5
:1037B000860280646AC00E94F30980918602806854
:1037C00064C0846062C081603DC0809186028E7F4B
:1037D0005CC0809186028D7F58C08091860216C0A1
:1037E0008091870218C0809187028D7F2BC08091C5
:1037F00086028F7E4AC0809186028F7D46C080916E
:1038000086028F7B42C080918602877F8B7F3DC07E
:10381000809187028D7F8E7F15C08091860282FB0A
:10382000222720F991E0922790FB82F990FB83F9FF
:103830002CC080918702982F909591708E7F892B54
:1038400090FB81F98093870222C00E94F309809146
:10385000860287FB222720F991E0922790FB87F9C7
:1038600014C081E00E94E21012C08091860284FBA5
:10387000222720F991E0922790FB84F906C08091DD
:103880008602982F909590FB80F980938602809114
:103890008602909187020E9452100E94F30980E0F4
:1038A00001C081E0DF91CF910895893289F1F0F470
:1038B000843171F1B0F4873009F077C081E08093F2
:1038C000240184E1809323018AE0809322018EE128
:1038D0008093210188E080931E0188E280931D017E
:1038E00064C092EE980F9A30F0F05FC0803509F412
:1038F00044C028F48F3409F058C08AE03FC08135B5
:1039000029F0823509F051C081E038C08FEF36C010
:1039100080916602882379F1109266021092650206
:103920001092640242C08D5180936602833099F0F8
:1039300038F4813069F08230D9F483E291E00DC02F
:10394000853099F078F0863099F48DE191E005C0EA
:1039500084E291E002C082E291E09093650280935C
:10396000640223C081E291E0F8CF8EE191E0F5CFCF
:10397000109266021AC080E0089586EFE09164021A
:10398000F0916502309789F02081082E000C990B88
:10399000820F911D8F3F910519F014F08FEF04C035
:1039A00097FF02C0108201C0808381E008950F93C9
:1039B0001F9341E050E060E070E08A019B0104C089
:1039C000000F111F221F331F8A95D2F7C901B801BA
:1039D0000E944B0A1F910F910C94F3098B3109F44B
:1039E00068C058F58B3009F486C078F4863009F445
:1039F00045C020F4853009F44BC07FC0873009F4FE
:103A00004AC0883009F477C078C0803109F464C0B6
:103A100068F48E3009F071C08091310282FB222758
:103A200020F991E0922790FB82F94CC0863109F48D
:103A300062C0893109F45FC060C08A32E1F060F48D
:103A4000873209F455C028F48E3108F456C08D51E0
:103A500050C08932E9F051C0833450F48A3308F001
:103A600045C0853309F444C0883309F444C045C0D7
:103A70008334F1F142C00E94D6103DC080913102E2
:103A8000817F8E7F8093310281E080936702089569
:103A90000E94C50530C080913102982F9095917099
:103AA00090FB80F980933102911125C0897F877F37
:103AB00010C08091310281FB222720F991E09227EA
:103AC00090FB81F9809331029923A9F08091310212
:103AD0008160809331020FC08091310283FB2227E5
:103AE00020F991E0922790FB83F9ECCF895301C034
:103AF00080E00E94D71C81E0089580E0089580E076
:103B000008950C947F1DCF93C82F80916702813058
:103B100069F038F08230C1F58C2F0E94551C81E08D
:103B200039C00E94460F8A3089F504C00E94460FB2
:103B30008A3061F48C2F0E94811D811104C08C2F6A
:103B40000E94EE1C1FC081E090E01CC08C2F0E94E0
:103B50007F1D811116C0C43189F058F4CB3089F033
:103B6000C031B1F482E08093670288E30E94551C63
:103B700008C0C93219F0C83321F00AC01092670298
:103B800007C081E0817006C01092670280E002C029
:103B900080E0F8CFCF910895CF93DF9386319C4595
:103BA00041F5EB010E94460F982F8A812091020176
:103BB00030910301882379F09A7A81E009F480E05A
:103BC00080936802911102C069E201C065E3C901F6
:103BD0000E9428210AC080916802811102C069E216
:103BE00001C065E3C9010E942A210E94880F80E07C
:103BF00001C081E0DF91CF9108950F931F93CF9380
:103C0000DF93C42FD22FFC0182818823C9F0409317
:103C10006B020E94CF2190936A028093690280E236
:103C20008C0F883008F057C0C77081E001C0880F42
:103C3000CA95EAF7DF91CF911F910F910C9450072D
:103C400080916B02481330C08091690290916A02A2
:103C50000E94E721883C910538F510E21D0FCD1731
:103C6000B9F080E28C0F883040F4C77081E001C069
:103C7000880FCA95EAF70E945707183028F581E0A7
:103C80009D2F977001C0880F9A95EAF70E94500700
:103C9000802F0E9447071830F0F4D77081E001C0F0
:103CA000880FDA95EAF70AC080E28C0F883098F422
:103CB000C77081E001C0880FCA95EAF7DF91CF9104
:103CC0001F910F910C945707802FDF91CF911F9177
:103CD0000F910C944707DF91CF911F910F91089599
:103CE0000F939C01CB01243F4CE5340731F188F45C
:103CF000293DFCE53F07D9F02A3D4CE5340779F131
:103D0000283D3C45A9F506E221EE41EE68ED7CE553
:103D10002BC0263FFCE53F07E1F0A8F0273F3C45DC
:103D200039F507E225EE46EE67EF7CE51DC007E2B8
:103D300025EE45EE69ED7CE517C006E221EE40EE8A
:103D400064EF7CE511C007E225EE44EE65EF7CE50B
:103D50000BC006E221EE42EE66EF7CE505C008E20C
:103D600021E045EE6AED7CE50E94FD1D80E008C083
:103D7000FC018281882319F010926B0201C081E05E
:103D80000F9108958EE1489B02C08150E1F7489B56
:103D9000FECF0895589880E28A95F1F7589A0895D1
:103DA000FC012AE02A95F1F728E090E080E031E07C
:103DB00040E14A95F1F7880F489B02C08160932744
:103DC00000C0000040E14A95F1F7215089F720E159
:103DD0002A95F1F729B100C0000030E13A95F1F7DA
:103DE000217092272081920F90830895EF92FF9285
:103DF0000F931F93CF93DF931F92CDB7DEB7198236
:103E00008C017C01E60EF11C0E151F0551F00E947D
:103E1000C21ECE0101960E94D01EF80181938F012F
:103E2000F3CF81E09981911180E00F90DF91CF91E4
:103E30001F910F91FF90EF900895509A589A08950E
:103E40005098589AE89AE9E6F0E080818C7F808368
:103E50000895615091E001C0990F6A95EAF720E05A
:103E600031E0992361F0492F482319F0589A23270C
:103E700001C0589840E24A95F1F79695F2CF222377
:103E800011F0589A01C0589880E28A95F1F7589835
:103E90000895FF920F931F93CF93DF93EC018C0152
:103EA000060F111DC017D10741F0F9900E94CA1EDC
:103EB00068E08F2D0E94291FF5CFDF91CF911F91D0
:103EC0000F91FF9008951F920F920FB60F92112439
:103ED0000F931F932F933F934F935F936F937F9312
:103EE0008F939F93AF93BF93EF93FF93CF93DF9302
:103EF0001F92CDB7DEB719820E94C21ECE01019675
:103F00000E94D01E082F069506950695902F96952F
:103F10009570202F2570920F292F237096959695D6
:103F2000920F877089135FC0898181115CC0043052
:103F300008F059C080E18A95F1F7589A509A82E0CA
:103F40008A95F1F700C0589888E0089F80011124F5
:103F5000D801AB5FBE4F1696ED91FC911797309745
:103F6000A9F06091A0017091A10114962D913C914E
:103F70001597260F371F11968D919C911297680FF8
:103F8000791F13964C9113978C910995F801EB5F6B
:103F9000FE4F6381662351F08091A0019091A101B1
:103FA00024813581820F931F0E94491F0E94CA1EDF
:103FB00080E18A95F1F758985098589A80E18A954F
:103FC000F1F7F801EB5FFE4F6081662351F08091BD
:103FD000A0019091A10121813281820F931F0E9443
:103FE000F61E0E94C21E0F90DF91CF91FF91EF91BC
:103FF000BF91AF919F918F917F916F915F914F9101
:104000003F912F911F910F910F900FBE0F901F9016
:1040100018950F931F93CF93DF93843091050CF085
:104020006DC0EC01F894509A589885E08A95F1F7A4
:1040300000009C2F969595702C2F2570920F892F3C
:1040400083709695969523E0CC0FDD1F2A95E1F7B6
:10405000980F8E01092B0E94CA1E84E08A95F1F701
:1040600000C068E0802F0E94291F80E18A95F1F747
:104070005098589A489902C000C0FCCF87E090E061
:10408000489B08C0019721F4509A589A789436C0FA
:1040900000C0F6CFFE01EB5FFE4F6381662381F027
:1040A0008091A0019091A10124813581820F931FFD
:1040B0000E94F61E811104C0509A589A78941FC02D
:1040C0000E94C21E80E28A95F1F75898509A80E1CA
:1040D0008A95F1F7CB5FDE4F6881662351F08091BE
:1040E000A0019091A10129813A81820F931F0E9422
:1040F000491F0E94CA1E789481E001C080E0DF91D0
:10410000CF911F910F9108959093A3018093A201E5
:104110000895909372028093710208950E9426166A
:10412000811103C080916C020895E0917102F091B9
:104130007202309721F00190F081E02D099480E027
:104140000895E0917102F0917202309721F002809F
:10415000F381E02D09940895E0917102F0917202CB
:10416000309739F022E0DC012C930480F581E02DBA
:104170000994089520916F02309170022817390731
:1041800071F09093700280936F02E0917102F09150
:104190007202309721F00680F781E02D099408958E
:1041A00020916D0230916E022817390771F09093BB
:1041B0006E0280936D02E0917102F091720230976D
:1041C00021F00084F185E02D09940895FC013296D8
:1041D00097E080E0915029F021912223D9F38F5F5D
:1041E000F9CF0895662349F0FC0132960896219193
:1041F000621729F0E817F907D1F780E0089581E008
:1042000008959C01FC0132969FEF80E04191461792
:1042100089F09F3F19F4411101C0982F8F5F8630BC
:10422000A9F79F3F39F0F901E90FF11D97FDFA95C4
:104230006283089508959C012A5F3F4FFC014281EB
:10424000461301C01282019682179307B9F70895A9
:104250000C9401210C941B21029626E0FC01119282
:104260002A95E9F7089508950C94332183E080930B
:1042700073020C943421811102C081E001C082E0FC
:10428000809373020C9434210C943B2181E0809341
:1042900073020C9434210C94462108950C944D2102
:1042A0000C944E210C944D210C944D210C944D21D5
:1042B000CF930E9454210E9490150E945221C0E089
:1042C0008C2F0E943E14892B29F4CF5FC630C1F792
:1042D00080E001C081E0CF91089508951F920F9270
:1042E0000FB60F9211248F939F93AF93BF9380913A
:1042F0007402811113C08091A2029091A302A09137
:10430000A402B091A5024196A11DB11D8093A20205
:104310009093A302A093A402B093A502BF91AF9182
:104320009F918F910F900FBE0F901F9018958091C5
:10433000AA02843031F10E9426061092740220E411
:1043400088E190E00FB6F894A895809360000FBEC6
:104350002093600083B7817F846083BF83B78160CF
:1043600083BF7894889583B78E7F83BF0FB6F89408
:10437000A895809160008861809360001092600031
:104380000FBE08950E94F3090C942A0682E084BDB2
:1043900093E095BD9AEF97BD80936E0008952FB777
:1043A000F8948091A2029091A302A091A402B091EE
:1043B000A5022FBF08952FB7F8946091A2027091C3
:1043C000A3028091A4029091A5022FBF08959C01A1
:1043D0004FB7F8948091A2029091A302A091A402F9
:1043E000B091A5024FBF821B930B0895CF92DF922D
:1043F000EF92FF922FB7F894C090A202D090A30240
:10440000E090A402F090A5022FBFA7019601261B01
:10441000370B480B590BCA01B901FF90EF90DF90A1
:10442000CF90089578941F920F920FB60F92112497
:104430008F939F93AF93BF938091A2029091A30219
:10444000A091A402B091A5020196A11DB11D809377
:10445000A2029093A302A093A402B093A502BF91DD
:10446000AF919F918F910F900FBE0F901F90189555
:10447000F89481E08093E00080E28093D800E9EC3A
:10448000F0E010828FE19EE40197F1F700C0000098
:104490001DBA109268001CBC10BE1FBA10927A00A0
:1044A00010926E0010926F001092710010927200C4
:1044B0001082ECEBF0E0108214B817B81AB81DB8EF
:1044C00010BA108215B818B81BB81EB811BA0C94DF
:1044D000003F0895809180020895089522E020937E
:1044E000E9002FEF3091E800215035FD06C035ED91
:1044F0003A95F1F700002111F5CF2091E80025FF52
:104500000BC040E050E066E070E00E94982480918B
:10451000E8008E778093E8000895CF93DF9321E041
:104520002093E9002FEF3091E800215035FD06C0BF
:1045300035ED3A95F1F700002111F5CF2091E80013
:1045400025FF14C0EC0140E050E068E070E00E94FC
:1045500098248091E8008E778093E80088E0FE013F
:10456000A8E7B2E001900D928A95E1F7DF91CF9133
:10457000089580937502709377026093760280911C
:10458000AA02843001F582E08093E9008FEF9091D8
:10459000E800815095FD06C095ED9A95F1F7000071
:1045A0008111F5CF8091E80085FF0DC040E050E01B
:1045B00063E070E085E792E00E9498248091E80033
:1045C0008E778093E8000895BC0184E00C94B922B2
:1045D000BC0183E00C94B9228091A902811109C029
:1045E0000E9429260E9486268091E20084608093A2
:1045F000E20008951092A90208950C944B21609155
:10460000A60281E0611101C080E00C9436219091F6
:10461000AA0281E0943009F080E06091A6020C9437
:104620003B2142E061EC81E00E94A22542E261EC84
:1046300082E00E94A2259091AA0281E0943009F0C4
:1046400080E06091A6020C9444218091AC028330FA
:1046500009F461C030F4813071F0823009F49AC0FD
:1046600008958A3009F486C08B3009F46CC0893013
:1046700009F0A8C020C08091AB02813A09F0A2C025
:104680008091E800877F8093E8008091AF0290914D
:10469000B002892B21F468E088E792E003C060E073
:1046A00080E090E070E00E94E3248091E8008B7746
:1046B0008093E80008958091AB02813209F082C0B6
:1046C0008091AF029091B002029708F07BC0809178
:1046D000E800877F8093E8008091E80082FD05C0B4
:1046E0008091AA028111F8CF6DC02091F3008091D2
:1046F000F20090E0922B029731F48091F10081302A
:1047000011F0863021F48091F10080938002809135
:10471000E8008B7753C08091AB02813A09F052C018
:104720008091AF029091B002892B09F04BC080912B
:10473000E800877F8093E8008091E80080FFFCCF4D
:104740008091310136C08091AB028132D9F58091E0
:10475000AF029091B002892BA9F58091E800877F84
:104760008093E8000E94D7258091AD0280933101AB
:104770000C94F3098091AB02813221F58091E8001D
:10478000877F8093E8000E94D7258091AE028093B6
:10479000810208958091AB02813AA1F48091E800F2
:1047A000877F8093E8008091E80080FFFCCF8091B4
:1047B00081028093F1008091E8008E778093E80079
:1047C0000C94D725089584B7877F84BF0FB6F894DB
:1047D000A8958091600088618093600010926000CD
:1047E0000FBE90E080E80FB6F8948093610090933C
:1047F00061000FBE0C9446210E9429260E94862645
:10480000E2EEF0E080818460808378940C941B2930
:1048100085E291E00C9489208091AA028530A9F468
:104820008091AA02853079F40E9497218091A80294
:104830008823B1F30E945821882391F30E94822497
:104840000E94F309EDCF0C94C221089508950C94B1
:104850002924292F332723303105C9F060F4213072
:10486000310581F02230310509F044C08BE390E03E
:104870002EE638E043C021323105E1F02232310525
:1048800049F138C082E190E029EA38E037C0992741
:104890008130910549F028F0029761F5E4E0F8E0F5
:1048A00005C0EAE6F8E002C0E8E4F8E0849190E0B0
:1048B0009F0124C06115710541F061307105D1F48B
:1048C00089E090E029E938E019C089E090E020E82B
:1048D00038E014C06115710541F06130710551F483
:1048E0008BE790E02BEB38E009C080E490E026E312
:1048F00039E004C080E090E020E030E0FA0131834C
:104900002083089580E189BD82E189BD09B400FE5C
:10491000FDCF8091D8008F7D8093D8008091E000FA
:1049200082608093E0008091E00081FDFCCF0895DB
:10493000CF92DF92EF92FF920F931F93CF93DF936B
:10494000EC018B017A010E94F625811133C0E1143C
:10495000F10439F0F70180819181081B190BC80F10
:10496000D91FC12CD12C0115110519F18091E80036
:1049700085FD16C08091E8008E778093E800E114F1
:10498000F10449F0F70180819181C80ED91ED182CE
:10499000C08285E00FC00E94F625882321F30AC05B
:1049A00089918093F10001501109FFEFCF1ADF0ABE
:1049B000DACF80E0DF91CF911F910F91FF90EF90C0
:1049C000DF90CF9008952091B1023091B202261766
:1049D000370748F06115710539F42091E8002E770A
:1049E0002093E80001C0B901FC0120E061157105C8
:1049F00079F18091AA028823F1F18530F1F180915B
:104A0000E80083FD3CC08091E80082FD2EC08091CB
:104A1000E80080FFEBCF2091F3008091F20090E05E
:104A2000922B6115710551F08830910538F4219170
:104A30002093F100615071090196F3CF21E00897AE
:104A400009F020E08091E8008E778093E800CECFD7
:104A50002111CFCF0AC08091AA02882361F085304E
:104A600061F08091E80083FD0AC08091E80082FF38
:104A7000F2CF80E0089582E0089583E0089581E018
:104A800008952091B1023091B2022617370748F0FD
:104A90006115710539F42091E8002E772093E80024
:104AA00001C0B901FC0120E06115710591F180910F
:104AB000AA02882309F440C0853009F43FC08091E0
:104AC000E80083FD3DC08091E80082FD2FC0809109
:104AD000E80080FFE9CF2091F3008091F20090E0A0
:104AE000922B6115710559F08830910540F424919D
:104AF0002093F1003196615071090196F2CF21E0C7
:104B0000089709F020E08091E8008E778093E80014
:104B1000CBCF2111CCCF0AC08091AA02882361F0AB
:104B2000853061F08091E80083FD0AC08091E80043
:104B300082FFF2CF80E0089582E0089583E0089537
:104B400081E00895982F973068F59093E9009817C1
:104B500039F07091EC002091ED005091F00003C00D
:104B6000242F762F50E021FD02C09F5FECCF3091C3
:104B7000EB003E7F3093EB003091ED003D7F3093B2
:104B8000ED003091EB0031603093EB007093EC005E
:104B90002093ED005093F0002091EE0027FDE5CF2B
:104BA00080E008958F708093E90081E008958091FE
:104BB000AB0287FF11C08091E80082FD05C08091A3
:104BC000AA028111F8CF11C08091E8008B770BC049
:104BD0008091AA02882349F08091E80080FFF8CFF5
:104BE0008091E8008E778093E80008952091E4009A
:104BF0003091E50095E64091EC00842F817040FFF4
:104C000023C08091E80080FD1DC08091AA02882306
:104C100099F0853099F08091EB0085FD11C04091AD
:104C2000E4005091E5002417350729F3915011F065
:104C30009A01E1CF84E0089582E0089583E0089529
:104C400081E0089580E008954091E80042FFDDCFC3
:104C500008950E9497260E949F26E0EEF0E0808152
:104C600081608083E8EDF0E080818F77808319BCDC
:104C7000A7EDB0E08C918E7F8C9380818F7E8083B6
:104C80001092A90208950F931F93CF93DF930E9470
:104C900097260E949F26C8EDD0E088818F77888371
:104CA00088818068888388818F7D888319BC109271
:104CB000AA021092A6021092A8021092A70200EE79
:104CC00010E0F80180818B7F8083888181608883F8
:104CD00042E060E080E00E94A225E1EEF0E0808109
:104CE0008E7F8083E2EEF0E080818160808380812E
:104CF00088608083F80180818E7F808388818061D5
:104D00008883DF91CF911F910F910895E8EDF0E036
:104D100080818F7E8083E7EDF0E0808181608083F9
:104D200084E082BF81E08093A9020C944326E8EDE1
:104D3000F0E080818E7F80831092E20008951092CF
:104D4000DA001092E10008951F920F920FB60F92B1
:104D500011242F933F934F935F936F937F938F9380
:104D60009F93AF93BF93EF93FF938091E10082FFF6
:104D70000BC08091E20082FF07C08091E1008B7F31
:104D80008093E1000E941A298091DA0080FF1FC001
:104D90008091D80080FF1BC08091DA008E7F8093C5
:104DA000DA008091D90080FF0DC080E189BD82E1E9
:104DB00089BD09B400FEFDCF81E08093AA020E9464
:104DC000EC2205C019BC1092AA020E94FA2280911E
:104DD000E10080FF19C08091E20080FF15C0809142
:104DE000E2008E7F8093E2008091E20080618093F8
:104DF000E2008091D80080628093D80019BC85E0E1
:104E00008093AA020E94FF228091E10084FF30C0BB
:104E10008091E20084FF2CC080E189BD82E189BDE0
:104E200009B400FEFDCF8091D8008F7D8093D8001B
:104E30008091E1008F7E8093E1008091E2008F7E7F
:104E40008093E2008091E20081608093E200809193
:104E5000A602882311F084E007C08091E30087FD5B
:104E600002C081E001C083E08093AA020E94072370
:104E70008091E10083FF29C08091E20083FF25C07B
:104E80008091E100877F8093E10082E08093AA0215
:104E90001092A6028091E1008E7F8093E1008091C4
:104EA000E2008E7F8093E2008091E2008061809337
:104EB000E20042E060E080E00E94A2258091F000E4
:104EC00088608093F0000E94FD22FF91EF91BF91D6
:104ED000AF919F918F917F916F915F914F913F9192
:104EE0002F910F900FBE0F901F9018951F920F9249
:104EF0000FB60F9211242F933F934F935F936F93AD
:104F00007F938F939F93AF93BF93CF93DF93EF9351
:104F1000FF93C091E900CF708091EC00D82FD17041
:104F200080FDD0E81092E9008091F000877F8093A7
:104F3000F00078940E94BA271092E9008091F00066
:104F400088608093F000CD2BCF70C093E900FF9173
:104F5000EF91DF91CF91BF91AF919F918F917F9111
:104F60006F915F914F913F912F910F900FBE0F90D6
:104F70001F9018951F93CF93DF93CDB7DEB7AA97F5
:104F80000FB6F894DEBF0FBECDBFEBEAF2E0809122
:104F9000F100819322E0E33BF207C9F70E94252349
:104FA0008091E80083FF2EC18091AB029091AC020A
:104FB000492F50E04A30510508F024C1FA01EE595A
:104FC000FF4F0C945C29803821F0823809F01AC117
:104FD00008C08091A7029091A802992389F082606D
:104FE0000FC08091AF028F70873008F00BC18093A3
:104FF000E9008091EB0085FB882780F91092E90099
:105000009091E800977F9093E8008093F1001092D0
:10501000F100D1C0282F2D7F09F0F4C0882319F0AA
:10502000823061F0EFC08091AD02813009F0EAC0BA
:10503000933009F080E08093A8022EC08091AD02E9
:1050400081112AC08091AF028F702FEF280F263078
:1050500008F0D8C08093E9002091EB0020FF1CC02D
:10506000933021F48091EB00806214C09091EB00AA
:1050700090619093EB0021E030E0A90102C0440F61
:10508000551F8A95E2F74093EA001092EA0080915A
:10509000EB0088608093EB001092E9008091E800BB
:1050A000877F8093E8000E94D725ACC08111AAC0F9
:1050B0001091AD021F778091E3008078812B80935F
:1050C000E3008091E800877F8093E8000E94D72565
:1050D0008091E80080FFFCCF8091E300806880939E
:1050E000E300111102C082E001C083E08093AA02B4
:1050F00089C08058823008F085C08091AD029091BF
:10510000AE028C3D53E0950779F583E08A838AE20D
:1051100089834FB7F894DE01139620E03EE051E218
:10512000E32FF0E050935700E49120FF03C0E29595
:10513000EF703F5FEF708E2F90E0EA3010F0C7966F
:1051400001C0C0968D939D932F5F243149F74FBFC7
:105150008091E800877F8093E8006AE270E0CE01EA
:1051600001960E94E32416C06091AF027091B002D4
:10517000AE014F5F5F4F0E942724BC01892B09F4C9
:1051800041C09091E800977F9093E80089819A81CF
:105190000E9441258091E8008B778093E80032C01F
:1051A000803881F58091E800877F8093E8008091C6
:1051B000A6028093F1008091E8008E7772CF811172
:1051C00021C08091AD029091AE0299270297D4F44C
:1051D0008091E800877F8093E8008091AD02809302
:1051E000A6020E94D7258091A602811106C0809157
:1051F000E30087FD02C081E001C084E08093AA0241
:105200000E9411238091E80083FF0AC08091E8008A
:10521000877F8093E8008091EB0080628093EB00B1
:10522000AA960FB6F894DEBF0FBECDBFDF91CF9127
:105230001F9108950895CF938091AA028823A1F029
:10524000C091E900CF709091EC00892F817090FDA2
:1052500080E8C82B1092E9008091E80083FD0E944D
:10526000BA27CF70C093E900CF9108950E942926F4
:105270001092AA020895E8EDF0E0808180618083B9
:105280008AE18A95F1F700C08091D9008170089574
:1052900097FB072E16F4009407D077FD09D00E94E3
:1052A000622907FC05D03EF4909581959F4F0895A3
:1052B000709561957F4F0895EE0FFF1F0590F49153
:1052C000E02D0994AA1BBB1B51E107C0AA1FBB1FFD
:1052D000A617B70710F0A61BB70B881F991F5A9582
:1052E000A9F780959095BC01CD010895FB01DC01E3
:1052F00004C08D910190801921F441505040C8F7AD
:10530000881B990B0895FB01DC0102C001900D92EE
:1053100041505040D8F70895F999FECF92BD81BD14
:10532000F89A992780B50895A8E1B0E042E050E0EE
:105330000C94C029262FF999FECF92BD81BDF89A11
:10534000019700B4021639F01FBA20BD0FB6F894C9
:10535000FA9AF99A0FBE08950396272F0E949B2967
:105360000E949A29252F0E949B29242F0C949B2967
:105370000196272F0E949B290C949A29DC01CB01CE
:10538000FC01F999FECF06C0F2BDE1BDF89A319655
:1053900000B40D9241505040B8F70895F894FFCFF3
:1053A000C80013020100000001000000000000001E
:1053B000060100000004070000000000002808505B
:1053C000011E0A14016A228D226E22E822E4226D57
:1053D0002201E200E900EA00B500B600B700CD0006
:1053E0008301CC008A01920194012102230224024C
:1053F0002502260227022A02B300B4006F007000C3
:10540000818283E200E900EA00B500B600B700CD72
:10541000008301CC008A019201940121022302241D
:10542000022502260227022A02B300B4006F007090
:105430000081828392F5F69697343536F7306667A9
:025440003A022E
:00000001FF
